:100000000C946D000C9495000C9495000C94950044
:100010000C9495000C9495000C9495000C9495000C
:100020000C9495000C9495000C9495000C949500FC
:100030000C9495000C9495000C9495000C949500EC
:100040000C9414050C9495000C9484050C945E0596
:100050000C9495000C9495000C9495000C949500CC
:100060000C94B6050C94950031333A32333A303063
:100070000046656220203420323032350000000016
:1000800000240027002A0000000000250028002B83
:1000900000000000002300260029000404040404DA
:1000A0000404040202020202020303030303030125
:1000B00002040810204080010204081020010204FC
:1000C00008102000000008000201000003040700DF
:1000D0000000000000000000D50611241FBECFEF75
:1000E000D8E0DEBFCDBF22E0A0E6B1E001C01D92A6
:1000F000A63FB207E1F711E0A0E0B1E0E6E9F8E1E0
:1001000002C005900D92A036B107D9F710E0CDE6F8
:10011000D0E004C02197FE010E941E0BCC36D1070F
:10012000C9F70E940E070C94490C0C940000089526
:100130000895833081F028F4813099F08230A9F05D
:1001400008958730A9F08830C9F08430B1F48091E7
:1001500080008F7D03C0809180008F778093800026
:10016000089584B58F7784BD089584B58F7DFBCFC6
:100170008091B0008F778093B00008958091B00097
:100180008F7DF9CFCF93DF93282F30E0F901ED5326
:10019000FF4F8491F901E155FF4FD491F901E556E4
:1001A000FF4FC491CC23A1F081110E949900EC2F44
:1001B000F0E0EE0FFF1FEF56FF4FA591B491EC91C9
:1001C000ED2381E090E009F480E0DF91CF91089584
:1001D00080E090E0FACF1F93CF93DF93282F30E099
:1001E000F901ED53FF4F8491F901E155FF4FD4918F
:1001F000F901E556FF4FC491CC23A9F0162F8111C8
:100200000E949900EC2FF0E0EE0FFF1FE957FF4F1F
:10021000A591B4918FB7F894EC91111108C0D095C5
:10022000DE23DC938FBFDF91CF911F910895DE2BEA
:10023000F8CFCF93DF9390E0FC01E155FF4F24917D
:1002400085569F4FFC0184918823D1F090E0880F60
:10025000991FFC01E358FF4FA591B491FC01E957A8
:10026000FF4FC591D49161110EC09FB7F8948C9146
:10027000E22FE0958E238C932881E223E8839FBFB1
:10028000DF91CF9108958FB7F894EC91E22BEC9326
:100290008FBFF6CF3FB7F8948091EF019091F001B6
:1002A000A091F101B091F20126B5A89B05C02F3FA6
:1002B00019F00196A11DB11D3FBFBA2FA92F982F8C
:1002C0008827BC01CD01620F711D811D911D42E087
:1002D000660F771F881F991F4A95D1F70895AF922F
:1002E000BF92CF92DF92EF92FF920F931F93CF9323
:1002F000DF936C017B018B01040F151FEB015E0185
:10030000AE18BF08C017D10759F06991D601ED9119
:10031000FC910190F081E02DC6010995892B79F7B8
:10032000C501DF91CF911F910F91FF90EF90DF906A
:10033000CF90BF90AF900895FC01538D448D252F31
:1003400030E0842F90E0821B930B541710F0CF966F
:10035000089501970895FC01918D828D981761F0A1
:10036000A28DAE0FBF2FB11D5D968C91928D9F5FB8
:100370009F73928F90E008958FEF9FEF0895FC0197
:10038000918D828D981731F0828DE80FF11D858D4A
:1003900090E008958FEF9FEF0895FC01918D228DDD
:1003A000892F90E0805C9F4F821B91098F73992762
:1003B000089589E492E00E94CD0121E0892B09F49F
:1003C00020E0822F089580E090E0892B29F00E94A0
:1003D000D90181110C9400000895FC01A48DA80F8F
:1003E000B92FB11DA35ABF4F2C91848D90E0019677
:1003F0008F739927848FA689B7892C93A089B18997
:100400008C91837080648C93938D848D981306C037
:100410000288F389E02D80818F7D80830895EF929B
:10042000FF920F931F93CF93DF93EC0181E0888FAE
:100430009B8D8C8D98131AC0E889F989808185FF7E
:1004400015C09FB7F894EE89FF896083E889F98920
:1004500080818370806480839FBF81E090E0DF9122
:10046000CF911F910F91FF90EF900895F62E0B8D75
:1004700010E00F5F1F4F0F731127E02E8C8D8E1130
:100480000CC00FB607FCFACFE889F989808185FF97
:10049000F5CFCE010E94ED01F1CFEB8DEC0FFD2FDA
:1004A000F11DE35AFF4FF0829FB7F8940B8FEA8952
:1004B000FB8980818062CFCFCF93DF93EC01888D61
:1004C0008823B9F0AA89BB89E889F9898C9185FDCF
:1004D00003C0808186FD0DC00FB607FCF7CF8C915D
:1004E00085FFF2CF808185FFEDCFCE010E94ED0127
:1004F000E9CFDF91CF910895FC01908190539A301C
:1005000008F090E0818180532AE0929F800D1124B1
:10051000089520918101260F3327331F21323105A1
:10052000ECF420911F02FC0190E080E0243069F09F
:1005300082E00895A09181012191AC014F595E4F55
:10054000A40FB52FB11D2C930196861798F38091B7
:100550008101680F6093810180E0089581E0089532
:1005600010921F0281E080931E021092F90161E057
:1005700082E10E94EB0061E083E10E94EB00E9EB85
:10058000F0E080818E7F808380818D7F808388E40E
:100590008093B80085E48093BC000895CF93DF93E7
:1005A00091E0909360018823B9F0C091B800D09198
:1005B000BA008091BC008A7B8093BC0060E082E13D
:1005C0000E94EB0060E083E10E94EB000E94B00219
:1005D000D093BA00C093B800DF91CF9108958F9265
:1005E0009F92AF92BF92CF92DF92EF92FF920F93C2
:1005F0001F93CF93DF93D0914802D13208F0D7C038
:10060000182FC09147020E944A016B017C01809122
:100610001F0281116BC082E080931F0210931E02A3
:100620008FEF80931D0210921C02D0931B02A7E251
:10063000B2E0EBEFF1E080E0D81391C01092FA0144
:100640008091FA01CC0FC82BC093FA018091F90177
:10065000813009F088C01092F9010E944A016B01B3
:100660007C018091FA018093BB00809121029091DE
:100670002202A0912302B0912402892B8A2B8B2B7A
:10068000A1F00E944A0100912102109122022091C2
:100690002302309124026C197D098E099F090617E7
:1006A00017072807390708F442C08091BC0083FD72
:1006B000D8CF85EC8093BC000E944A016B017C017D
:1006C00080911F02823009F450C080911D028F3F3B
:1006D00009F46FC080911D02803209F46CC08091D2
:1006E0001D02803309F469C084E026C08091210294
:1006F00090912202A0912302B0912402892B8A2B8F
:100700008B2B09F484CF0E944A01809021029090A3
:100710002202A0902302B09024026C197D098E0958
:100720009F0986169706A806B90608F070CF809133
:1007300020020E94CE0285E010922602109248020A
:1007400010922502DF91CF911F910F91FF90EF90B2
:10075000DF90CF90BF90AF909F908F9008959D9124
:1007600091938F5F69CF85EEA5CF80912102909103
:100770002202A0912302B0912402892B8A2B8B2B79
:1007800009F49ECF0E944A01009121021091220299
:1007900020912302309124026C197D098E099F0952
:1007A000061717072807390708F08ACFC0CF81E05E
:1007B000C3CF80E0C1CF82E0BFCF83E0BDCF1F9326
:1007C000CF93DF93EA01122FDC0111968D919C915A
:1007D000DC01ED91FC910280F381E02D0995C817B1
:1007E000D90729F4812F0E94EF0291E0811190E056
:1007F000892FDF91CF911F910895CF93DF93EC0163
:100800008B818823A1F0888191E0909325028093C9
:100810004702109226021092480281E00E94EF02E5
:1008200091E0811190E0892FDF91CF91089510928E
:10083000F8011092F70110922602109248020E94CD
:10084000B00287E990E09093F4018093F30188E986
:1008500090E09093F6018093F50181E08B83CE01C7
:100860000E94FD03982F8111CECFDDCF0895E09136
:10087000F8018091F701E81730F4F0E0EC53FE4FF7
:10088000808190E008958FEF9FEF08959091F80197
:100890008091F7012FEF3FEF981748F4E92FF0E030
:1008A000EC53FE4F208130E09F5F9093F801C90127
:1008B00008958091F7019091F801891B990B089593
:1008C000CF92DF92EF92FF920F931F93CF93DF931C
:1008D0007C01CB018A0120912502222389F0EB01C2
:1008E0006B01C40ED51ECC15DD0569F06991D701E9
:1008F000ED91FC910190F081E02DC7010995F3CFB6
:10090000642F0E948902C801DF91CF911F910F913E
:10091000FF90EF90DF90CF900895CF93DF931F92D9
:10092000CDB7DEB76983209125022223F9F020910B
:100930004802203258F021E030E0FC01338322836A
:1009400090E080E00F90DF91CF9108958091260292
:10095000E82FF0E0E95DFD4F998190838F5F8093F0
:1009600026028093480281E090E0ECCF61E0CE0166
:1009700001960E948902F7CF90E080E00895CF931E
:10098000DF93FC0101900020E9F73197AF01481B8C
:10099000590BBC0189E492E00E946F01EC0142E036
:1009A00050E06AE271E089E492E00E946F018C0FEE
:1009B0009D1FDF91CF91089585ED8093BC008091BC
:1009C000210290912202A0912302B0912402079665
:1009D000A11DB11D23E0B695A795979587952A95FA
:1009E000D1F72091BC0024FD03C010921F0208958E
:1009F00040912102509122026091230270912402C1
:100A0000452B462B472B69F30097A105B10541F013
:100A10002AE22A95F1F700C00197A109B109E1CFB7
:100A2000809120020C94CE021F920F920FB60F926B
:100A300011242F933F938F939F93AF93BF938091F4
:100A4000EB019091EC01A091ED01B091EE0130919C
:100A5000EA0123E0230F2D3758F50196A11DB11DA2
:100A60002093EA018093EB019093EC01A093ED01B8
:100A7000B093EE018091EF019091F001A091F1010E
:100A8000B091F2010196A11DB11D8093EF019093E9
:100A9000F001A093F101B093F201BF91AF919F914A
:100AA0008F913F912F910F900FBE0F901F9018952F
:100AB00026E8230F0296A11DB11DD2CF1F920F92DF
:100AC0000FB60F9211242F933F934F935F936F9321
:100AD0007F938F939F93AF93BF93EF93FF9389E49B
:100AE00092E00E94ED01FF91EF91BF91AF919F9134
:100AF0008F917F916F915F914F913F912F910F90C7
:100B00000FBE0F901F9018951F920F920FB60F9265
:100B100011242F938F939F93EF93FF93E0915902AA
:100B2000F0915A028081E0915F02F091600282FDB3
:100B30001BC09081809162028F5F8F73209163024E
:100B4000821741F0E0916202F0E0E75BFD4F958F84
:100B500080936202FF91EF919F918F912F910F905F
:100B60000FBE0F901F9018958081F4CF1F920F92A7
:100B70000FB60F9211242F933F934F935F936F9370
:100B80007F938F939F93AF93BF93EF93FF93809146
:100B9000B900887F803609F44AC0F0F5883209F43C
:100BA000A7C018F5803109F49BC0B8F4882309F474
:100BB000F9C0883009F494C0FF91EF91BF91AF91D3
:100BC0009F918F917F916F915F914F913F912F9165
:100BD0000F900FBE0F901F901895883109F488C0B0
:100BE000803251F780931D0214C0803409F49DC0F7
:100BF00040F48033B9F38833F9F680931D0285EC15
:100C0000B0C0803509F485C0883509F496C08834B1
:100C100099F60E94DC04D0CF883909F48CC038F5ED
:100C2000883729F050F4883611F0803729F683E0B0
:100C300080931F021092A30157C0883809F47BC02B
:100C4000803919F0803809F0B7CF8091A301803244
:100C500008F071C0E091A30181E08E0F8093A301A1
:100C60008091BB00F0E0ED57FE4F80833DC0803B9C
:100C700039F0E0F4803A09F479C0883A09F09CCF61
:100C800084E080931F021092820110928101E09112
:100C9000F301F091F40109958091810181110FC058
:100CA00081E0809381011092610109C0803C09F4C8
:100CB000A6CF883C09F4A3CF883B09F07DCFE09113
:100CC000820181E08E0F80938201F0E0EF59FE4FA8
:100CD00080818093BB00909182018091810129C025
:100CE0008091FA018093BB0085EC8093BC0064CFB7
:100CF00090911C0280911B02981758F5E0911C02FC
:100D000081E08E0F80931C02F0E0E550FE4F808161
:100D1000E9CFE0911C0281E08E0F80931C0280914C
:100D2000BB00F0E0E550FE4F808390911C02809163
:100D30001B029817C8F285E8D8CFE0911C0281E029
:100D40008E0F80931C028091BB00F0E0E550FE4FB7
:100D5000808380911E0281115CCF81E08093F90134
:100D600084EA8093BC0010921F0226CF85EC80930A
:100D7000BC0010921F028091A301803230F4E091F8
:100D8000A301F0E0ED57FE4F10826091A30170E0E7
:100D9000E091F501F091F60183E891E00995109258
:100DA000A3010ACF10921D0234CFE9E4F2E01382CE
:100DB000128288EE93E0A0E0B0E084839583A6835E
:100DC000B7832AE031E03183208325EC30E035879A
:100DD000248724EC30E03787268720EC30E0318B05
:100DE000208B21EC30E0338B228B22EC30E0358BF2
:100DF000248B26EC30E0378B268B118E128E138ECF
:100E0000148EE6EEF2E01382128284839583A68329
:100E1000B7838CE191E0918380830895CF93DF9332
:100E2000CDB7DEB72B970FB6F894DEBF0FBECDBFA0
:100E3000789484B5826084BD84B5816084BD85B5B5
:100E4000826085BD85B5816085BD80916E008160C1
:100E500080936E0010928100809181008260809367
:100E60008100809181008160809381008091800069
:100E70008160809380008091B10084608093B10094
:100E80008091B00081608093B00080917A0084608E
:100E900080937A0080917A00826080937A008091BA
:100EA0007A00816080937A0080917A0080688093D4
:100EB0007A001092C100E0915902F0915A0282E04A
:100EC0008083E0915902F0915A021082E09155021C
:100ED000F09156021082E0915702F091580280E1A1
:100EE000808310926102E0915D02F0915E0286E0E3
:100EF0008083E0915B02F0915C028081806180835D
:100F0000E0915B02F0915C02808188608083E091D7
:100F10005B02F0915C02808180688083E0915B02DB
:100F2000F0915C0280818F7D80838091E8019091B7
:100F3000E901009711F00E94C00B86E090E00E944A
:100F4000240B7C0188E6D7018C9386EE92E0129602
:100F50009C938E93119713961C92139780E290E0C6
:100F600015969C938E931497F092E901E092E80114
:100F70001092F8011092F701109226021092480286
:100F80000E94B00287E990E09093F4018093F3010E
:100F900088E990E09093F6018093F50181E0F701F4
:100FA0008383C7010E94FD03811105C08DE291E09A
:100FB0000E94BF04FFCF8FE391E00E94BF0460E076
:100FC0008FE00E94190160E08EE00E94190161E04B
:100FD0008AE00E94190161E089E00E94190161E044
:100FE0008EE00E94EB0061E08FE00E94EB0060E089
:100FF0008AE00E94EB0060E089E00E94EB0080E262
:1010000090E00E94FC0AB4EACB2EB1E0DB2E560140
:1010100000E2E02EF12C80528E3588F4F0E4EF16D9
:10102000F10469F0C7010E94FC0AD5018D935D01AE
:10103000BFEFEB1AFB0AC7010E94FC0AECCFF701D5
:10104000EC57FE4F1082E4EAF1E001900020E9F74E
:10105000ED5AF14009F0BFC0E6E4F1E08EE491E022
:101060003191D6012D916D013213B5C08E179F07B6
:10107000B9F777E0872E912C65EC262E3324339434
:101080001982C090E801D090E901D60114968D91A3
:101090009C911597892B09F408C28C9130922502F6
:1010A00080934702109226021092480220E041E00D
:1010B00050E0BE016F5F7F4FC6010E94DF038823AF
:1010C00009F4F3C1F12CE12CF601848195818401AE
:1010D0000E191F098017910708F48C01D601AC90F6
:1010E0000E944A012B013C0180911F02811165C1C0
:1010F000B02EB0E2B01710F450E2B52E30921F02BD
:1011000021E0C401801B910BE816F90608F420E0E9
:1011100020931E02EFEFE0931D0210921C028FEF4E
:101120008B0D80931B023092FA018091FA01AA0C78
:10113000A82AA092FA018091F901813009F088C1B2
:101140001092F9010E944A012B013C018091FA01A1
:101150008093BB008091210290912202A0912302F2
:10116000B0912402892B8A2B8B2BA1F00E944A017B
:1011700020912102309122024091230250912402B9
:10118000641975098609970926173707480759070B
:1011900008F434C18091BC0083FDD8CF2092BC00FC
:1011A0000E944A012B013C0180911F02813009F409
:1011B00053C180911C028B1510F4B0901C02ABEF50
:1011C000B1E0E4ECF1E080E08B1509F41CC19D91E5
:1011D00091938F5FF9CFF12CE12C60E0C7010E9461
:1011E000040BBFEFEB1AFB0AE8E7EE16F104A9F7D0
:1011F000A0E2EA2EF12C60E0C7010E94040BFFEF91
:10120000EF1AFF0A20E4E216F104A9F7E6E4CE2E75
:10121000E1E0DE2EF0E2EF2EF12CD6016D916D01B2
:10122000662339F0C7010E94040BBFEFEB1AFB0ADB
:10123000F4CF4BE050E061E770E0FE0131967F01B2
:10124000CF010E94F30ACE010A960E947C02082F69
:10125000E981E154E33118F50E2E000CFF0BED5C33
:10126000F64F0C941E0BC5094F094F09D9094F09B8
:10127000DB094F094F094F0946094F094F09CC09AE
:10128000D709D5094F094F094F09D3098A8111E0C0
:10129000813629F08B8116E08E3609F017E0CE01F9
:1012A00005960E947C02D82E48E050E068E670E087
:1012B000C7010E94F30AC7010E947C02C82ECE011A
:1012C00004960E947C02B82ECE0107960E947C02F2
:1012D000382F86E0D7011D928A95E9F72AE0832FFF
:1012E000622F0E94120B982F880F890F880F830F8F
:1012F0008A838B2D0E94120B982F880F890F880FDD
:101300008B0D8B838C2D0E94120B982F880F890FC9
:10131000880F8C0D8C838D2D0E94120B982F880FB7
:10132000890F880F8D0D8E83812F0E94120B982FAD
:10133000990F890F880F180F1F83802F0E94120B9F
:10134000982F880F890F880F800F88878091E80178
:101350009091E901FC01248135812830310580F02C
:10136000208131E03093250220934702109226021B
:101370001092480221E048E050E0B7010E94DF03EC
:101380008FE491E00E94BF0474CE8B8114E0823719
:1013900009F485CF18E083CF8B8113E0823709F4FD
:1013A0007ECF15E07CCF19E07ACF1AE078CF1BE032
:1013B00076CF1CE074CF12E072CF80912102909121
:1013C0002202A0912302B0912402892B8A2B8B2B1D
:1013D00009F48ACE0E944A01209121023091220212
:1013E00040912302509124026419750986099709D6
:1013F000261737074807590708F076CE8091200254
:101400000E94CE02B12C1092F801B092F701B016F2
:10141000110609F04AC0AA24A394B12CAC0EBD1E3B
:10142000AE0CBF1C3501C5018619970980179107BD
:10143000A8F5D60111968D919C91DC01ED91FC915E
:101440000284F385E02D0995F50181935F01EBCFCF
:10145000F5EEF093BC00A4CE80912102909122027F
:10146000A0912302B0912402892B8A2B8B2B09F4A3
:101470009BCE0E944A01209121023091220240918C
:1014800023025091240264197509860997092617C9
:1014900037074807590708F087CEB0CFE00EF11E96
:1014A000F7E0EF16F10408F40FCE2A81822F90E0C6
:1014B00034E0959587953A95E1F7982F990F990F14
:1014C000891B880F820F31F08EE00E94C200892BA9
:1014D00009F07AC084E591E00E94BF0461E08AE0EF
:1014E0000E94EB0061E089E00E94EB002FB7F894C6
:1014F0008091EB019091EC01A091ED01B091EE0192
:101500002FBF8093E4019093E501A093E601B0938F
:10151000E7018FE00E94C200892BD9F72FB7F8941A
:101520008091EB019091EC01A091ED01B091EE0161
:101530002FBF4091E4015091E5016091E601709167
:10154000E701841B950BA60BB70B80319742A105D1
:10155000B105F8F260E08AE00E94EB0060E089E00B
:101560000E94EB000E944A016B017C0188E8482E32
:1015700083E1582E612C712C0E944A016C197D095F
:101580008E099F09683E734081059105A8F381E0AB
:10159000481A51086108710898EEC90E93E0D91EE7
:1015A000E11CF11C411451046104710429F7E0E0CD
:1015B000F0E0EF2B09F464CD0E94D901882309F4EF
:1015C0005DCD0E94000058CD8FE00E94C200892BA3
:1015D00029F061E08AE00E94EB00F6CF60E08AE04B
:1015E0000E94EB00E4CFFB01DC0102C005900D92EC
:1015F00041505040D8F70895F999FECF92BD81BD72
:10160000F89A992780B50895262FF999FECF1FBA29
:1016100092BD81BD20BD0FB6F894FA9AF99A0FBE1B
:1016200001960895991B79E004C0991F961708F058
:10163000961B881F7A95C9F780950895EE0FFF1FB6
:101640000590F491E02D09940F931F93CF93DF93AE
:101650008230910510F482E090E0E091F402F09184
:10166000F50230E020E0B0E0A0E0309799F42115D9
:10167000310509F44AC0281B390B24303105D8F54F
:101680008A819B816115710589F1FB0193838283B6
:10169000FE0111C040815181028113814817590711
:1016A000E0F04817590799F4109761F012960C93DF
:1016B000129713961C933296CF01DF91CF911F9111
:1016C0000F9108950093F4021093F502F4CF2115C1
:1016D000310551F04217530738F0A901DB019A0197
:1016E000BD01DF01F801C1CFEF01F9CF9093F50201
:1016F0008093F402CDCFFE01E20FF31F819391930B
:101700002250310939832883D7CF2091F2023091BA
:10171000F302232B41F42091020130910301309315
:10172000F3022093F2022091000130910101211572
:10173000310541F42DB73EB74091040150910501A8
:10174000241B350BE091F202F091F302E217F3074C
:10175000A0F42E1B3F0B2817390778F0AC014E5F21
:101760005F4F2417350748F04E0F5F1F5093F30269
:101770004093F202819391939FCFF0E0E0E09CCF01
:10178000CF93DF930097E9F0FC0132971382128226
:10179000A091F402B091F502ED0130E020E0109745
:1017A000A1F420813181820F931F2091F2023091A8
:1017B000F3022817390709F061C0F093F302E093B0
:1017C000F202DF91CF910895EA01CE17DF07E8F525
:1017D0004A815B819E0141155105B1F7E901FB8307
:1017E000EA8349915991C40FD51FEC17FD0761F4A5
:1017F000808191810296840F951FE90199838883E6
:10180000828193819B838A83F0E0E0E012968D9140
:101810009C9113970097B9F52D913C911197CD01AB
:101820000296820F931F2091F2023091F302281743
:10183000390739F6309751F51092F5021092F402FB
:10184000B093F302A093F202BCCFD383C283408152
:101850005181840F951FC817D90761F44E5F5F4F00
:1018600088819981480F591F518340838A819B81C8
:10187000938382832115310509F0B0CFF093F502EF
:10188000E093F4029ECFFD01DC01C0CF13821282EF
:06189000D7CFF894FFCF52
:101896000000F6028000000000000F026F019C01AC
:1018A6005C02CD01AB01BF01000000008D046004A5
:1018B600BC0436045904460437040D0A00436F7508
:1018C6006C646E27742066696E6420525443004827
:1018D6006F6C6121210031333A32333A3030006F78
:1018E6006B21210041627269656E646F2E2E2E0097
:00000001FF
